:020000040800F2
:100000000080002073380008D5370008E938000860
:10001000D9370008DB370008DD3700080000000092
:10002000000000000000000000000000DF370008B2
:10003000E137000800000000E3370008E90D000880
:10004000E7370008E9370008EB370008ED3700080C
:10005000EF370008F1370008F3370008F5370008DC
:10006000F7370008F9370008FB370008FD370008AC
:10007000FF37000801380008033800080538000879
:10008000073800080000000009380008011B0008BC
:10009000E51B00080F380008113800081338000865
:1000A0001538000817380008193800081B380008F0
:1000B0001D3800081F3800082138000823380008C0
:1000C0002538000827380008293800082B38000890
:1000D0002D3800082F380008313800083338000860
:1000E0003538000837380008393800083B38000830
:1000F0003D3800083F380008413800080000000083
:1001000000000000433800080000000045380008E7
:100110004738000800000000493800084B38000844
:100120004D3800084F38000851380008533800088F
:100130005538000800000000000000005738000893
:10014000593800085B38000800000000000000007B
:10015000000000000000000000000000000000009F
:100160000000000000000000000000005D380008F2
:100170005F380008000000000000000000000000E0
:1001800000000000613800080000000000000000CE
:10019000000000000000000000000000000000005F
:1001A0000000000000000000633800086538000807
:1001B00067380008693800086B3800080000000044
:1001C000000000006D380008000000000000000082
:0801D0006F38000871380008C7
:1001D80008B5544B9A6D42F080529A651A6842F4F9
:1001E80080321A6000234F490A68013312F4003F35
:1001F80015D1B3F5A02FF7D14A4A116821F48031FF
:100208001160116841F48071116011460A68013368
:1002180012F4806F41D1B3F5A02FF7D33CE0424BE5
:1002280040F202721A60A3F580539A689A609A683D
:100238009A609A689A604FF44062DA60D3F888202E
:1002480022F04062C3F88820D3F8882042F0006288
:10025800C3F88820DA6842F08872DA60DA6842F017
:100268000302DA601A6842F080721A601A4613684C
:1002780013F0007FFBD02B4A936843F0030393608D
:10028800936803F00C030C2BFAD101F005FF254A03
:10029800936C43F48073936408BD234B40F202725D
:1002A8001A60A3F580539A689A609A689A609A6867
:1002B8009A601022DA604FF44062DA60DA68DA6035
:1002C800DA68DA60D3F8882022F04062C3F8882020
:1002D800D3F8882042F00062C3F88820DA6842F038
:1002E8008872DA60DA6842F00202DA601A6842F06C
:1002F80080721A601A46136813F0007FFBD0094A0F
:10030800936843F003039360936803F00C030C2B8A
:10031800FAD101F0C1FE034A936C43F480739364ED
:0C032800BAE700BF0010024000200240B5
:100334004FF090434FF080729A61024BC8221A60CA
:08034400704700BFD01A002031
:10034C00332303494AF6AA220A60013BFCD17047C9
:04035C00003000402D
:1003600010B5524BDB6913F0800F0BD0504A136865
:100370005049C85C4D498862013313604E4A126887
:10038000934222D24D4B1B68F3B94C4B14221A6096
:100390004B4B4AF6AA221A604A4B1B68C3B94A4B18
:1003A0001B683BB3072B16D84FF090424FF4807177
:1003B00091610133444A1360444B1B780133DBB233
:1003C000042B21D8414A137010BD01F027FFD9E753
:1003D00002F0F4F8E3E74FF090424FF08071916142
:1003E00001330B2B03D9384B01221A60E4E7364A5C
:1003F0001360E1E7364B1B68002BDDD14FF09043D3
:100400004FF480729A61D7E7304B00221A70314B5B
:100410001B684BB1304B1B6833B1304A1368591E0F
:100420001160023BFE2B08D82D4B1B780133DBB249
:10043000092B05D82A4A1370C6E702F00FF9F3E733
:10044000274B00221A70274B1B687BB94FF0904353
:100450001B6913F4804F0DD0234B1B68012BB3D1C4
:1004600000F0E8FC204B00221A600CE0522001F062
:10047000DBFDEBE71C4B1B68002BA5D100F0DAFC81
:10048000194B01221A6000F0DFFD184B41F288324F
:100490001A600B484AF6AA21154A1C4601601368E7
:1004A000002B91D12368002BF8D18DE70038014053
:1004B0005C1A00201C180020601A0020C41A0020BA
:1004C00000300040541A0020CC1A0020E71A002007
:1004D000D01A0020681A0020741A0020781A002010
:1004E0001A180020BC1A0020341A0020C01A00205C
:0404F000381A002096
:1004F400074B186058B170B5064E4AF6AA251C463B
:100504003560FFF72BFF2368002BF9D170BD7047CE
:08051400D41A00200030004061
:10051C0030B42249CC68E443214B1C600B69DB43AB
:10052C00204A13604A69D2431F4802608969C94353
:10053C0008D01A48C069C04304D01C4D29601C491E
:10054C00086007E0194940F283400860184945F2F9
:10055C00407008600F2C02D911490F20086063B954
:10056C00104B4FF400711960B2F51F7F03D30E4B83
:10057C0040F27B221A6030BC7047172B03D8094B12
:10058C0018211960F0E7074B1B68B3F5007FEBD916
:10059C00044B4FF400711960E6E700BF00400008FF
:1005AC00D81A0020601A0020581A0020801A002047
:0405BC00C81A002039
:1005C00010B50446574B186910F48030FBD1554BD9
:1005D0005B69002B23DA534B534A9A6002F188324D
:1005E0009A60A3F5F8334AF6AA221A604D4A1369B5
:1005F00013F4803FFBD14B4B4C4A5A615A6942F489
:1006000080325A61186910F48030FBD1454B1A6969
:1006100042F001021A611B6913F0020F00D010BDF5
:10062000404A536923F0020353611420FFF762FF2D
:100630003F4B9C426CD03B4A536943F001035361EA
:100640003C4A002313603C4B1B88DB435360354B13
:10065000186910F48030FBD1324B1A6942F0010264
:100660001A611B6913F0020FD9D1324A334B1B8830
:10067000DB439360324B1B68DB43D360294B186923
:1006800010F48030FBD1274B1A6942F001021A6145
:100690001B6913F0020FC2D1264A2A4B1B68DB43A9
:1006A0001361294B1B68DB4353611E4B186910F41F
:1006B0008030FBD11B4B1A6942F001021A611B69A1
:1006C00013F0020FABD11B4A1B4B1B88DB4393611A
:1006D0001A4B1B88DB43D361124B186910F480302E
:1006E000FBD1104B1A6942F001021A611B6913F029
:1006F000020F94D10B4B5A6922F001025A615A69D8
:1007000042F000425A610A20FFF7F4FE012086E71A
:10071000044A536943F0004353616420FFF7EAFE43
:1007200001207CE7002002402301674542000003CE
:10073000C9B3E7A500400008801A0020C81A0020AD
:0C074000D81A0020601A0020581A00206F
:10074C002DE9F04178B9204B03F50071002203F834
:10075C00012F8B42FBD1DFF874801B4D08F500761E
:10076C0044461B4F23E0431E9A0802F5803209329F
:10077C0003F00303580200EBC220164A02F5007482
:10078C001346801AC258D243110E1970110C5970AD
:10079C00110A9970DA700433A342F3D1DBE7601EBF
:1007AC00A0EB080080B201F0E5FDB4420AD00134A0
:1007BC0015F8013F22789A42F7D03A68002AEED118
:1007CC002370F2E7BDE8F081171600201B180020FB
:0807DC00581A00201816002035
:1007E400114A936D43F4003393654FF090431A68B4
:1007F40022F010021A601A6842F020021A601A6A83
:1008040022F470621A621A6A42F4E0621A62074BB6
:1008140040F2A112DA604FF400325A6000229A606A
:1008240009221A60704700BF0010024000440040D3
:10083400034AD36913F0800FFBD0014B98627047D1
:04084400004400402C
:100848002DE9F8430027934B9A6D42F080529A6540
:10085800DA6C42F00102DA64DA6C42F00202DA641D
:100868004FF090424FF0205313608B4B1F608B4921
:10087800D1604FF0AA32DA60FFF7AAFC884B142245
:100888001A60884B1F60884B1F60884B1F60884B1D
:100898001F60884B40F283421A60874B45F24072D2
:1008A8001A60864B1F60864B1F60864B1F60864B05
:1008B8004FF400721A60854B1F606423844A1360EA
:1008C800844A1360844B1B68844AA2FB03239B0958
:1008D800013BB3F1807F09D24FF0E0225361804B96
:1008E800F02183F823109761072313617D4C45F2AB
:1008F800555323604FF6FF73A3600220FFF7F6FD00
:1009080002206060FFF7F2FD4CF6CC4323604FF401
:10091800FA70FFF7EBFD744B00221A604FF090431A
:100928001B6913F4005F58D04FF09044236823F4F8
:1009380040332360236843F4803323604FF480738B
:10094800A361236823F040532360E36843F0805396
:10095800E360E36823F00053E3600A20FFF7C6FD75
:10096800564B00221A60236913F4804F02D1534B6F
:1009780001221A60FFF732FF1420FFF7B7FD40206D
:10098800FFF754FFFFF7C6FD0020FFF7DBFE0A2044
:10099800FFF7ACFD01F0C6FB01F03CFC0A20FFF7B5
:1009A800A5FD524B00221A6000F04AFB3F4B41F272
:1009B80088321A604D4C1D46FFF7CEFC236813B9E8
:1009C8002B68002BF8D10A20FFF790FD484B002236
:1009D8001A703A4C1D46354E10E04648FFF7ECFDBC
:1009E8004FF4FA70FFF782FD3F4B01221A609BE734
:1009F8002B7002F0DBFB08E002F0D8FBFFF7ACFC41
:100A08002368F3B928780028F2D100F0E5FE58B140
:100A1800C0B25A28F0D14FF47A733360364B0022B3
:100A28001A6001F033FCE9E73368002BE6D1274B65
:100A38001B68002BE2D00023244A13601C4A136071
:100A4800DCE700F0C9FE0028D8D05FFA80F9C0F3CF
:100A58000318B8F10D0F28BF4FF0000800F0BCFED6
:100A680080B1C7B2A8F10C03DBB2012B98BF0023F9
:100A78000AD8B8F1000FC1D03A464946404601F0BD
:100A8800D5FFBBE74FF0000800F0A6FE0028B5D060
:100A9800C3B2EEE70010024000040048AAAA01967B
:100AA800C41A0020D01A0020D41A0020C01A00202E
:100AB800CC1A0020801A0020C81A0020341A0020FE
:100AC800D81A0020581A0020601A0020441A002062
:100AD800481A00204C1A002008000020D34D62104C
:100AE80000ED00E000300040BC1A0020381A002059
:0C0AF800E61A0020C9B3E7A5541A00203C
:100B040070B5ADF5006D002800F09880431E9C0878
:100B140003F00303D80104F5803E0EF1090E4FEAF9
:100B2400CE2EF446ADF104030DF2FC750DF5006212
:100B3400C2F5006104310EEB03025258D24343F86C
:100B4400042FAB42F7D1484A002100EB91051678F7
:100B540053781B0443EA0663D6783343967843EA12
:100B640006234DF8253004310432B1F5007FECD171
:100B74003E4A136913F4803FFBD13C4B5B69002B65
:100B84006ADB3B4B4AF6AA221A60384A136913F40B
:100B9400803FFBD104F10903DB0043F0407343F0D1
:100BA4000203324A5361536943F480335361134659
:100BB4001C6914F48034FBD12C4B1A6942F00102F5
:100BC4001A611B6913F0020F3ED1284B5A6922F0B7
:100BD40002025A615A6942F001025A610EF500613B
:100BE4006B46A3EB0E0E0EF10405204B5EF80C20B1
:100BF400D243CCF8002055F80C20D243CCF8042082
:100C04000CF1080C1C6914F48034FBD11A6942F00D
:100C140001021A611A6912F0020F15D16145E5D17A
:100C2400124B5A6922F001025A615A6942F0004299
:100C34005A610A20FFF75CFC012405E00120FFF75C
:100C4400BDFC044620B1012420460DF5006D70BDA5
:100C5400084802F08AFFF7E7044B074A9A6002F15A
:100C640088329A608DE700BF1C18002000200240E3
:0C0C740000300040243B000823016745CD
:100C800010B5041E7ADB092C72D9632C64D9B4F533
:100C90007A7F56D342F20F739C4246D9404B9C4216
:100CA00037D9404B9C4228D93F4B9C421AD33F4BEB
:100CB0009C420CD93E4B9C4265D83E48A0FB043078
:100CC000400E3D4B03FB1044303001F0ADF93B4882
:100CD000A0FB0430800D344B03FB10443030C0B215
:100CE00001F0A2F93648A0FB0430800C354B03FB21
:100CF00010443030C0B201F097F96009324BA3FBC9
:100D00000030C009314B03FB10443030C0B201F059
:100D10008BF92F48A0FB0430400B42F2107303FB09
:100D200010443030C0B201F07FF92A48A0FB0430F3
:100D300080094FF47A7303FB10443030C0B201F0E5
:100D400073F92548A0FB04304009642303FB1044D9
:100D50003030C0B201F068F92048A0FB0430C00870
:100D600000EB8003A4EB43043030C0B201F05CF927
:100D700004F13000C0B201F057F910BD2D2001F090
:100D800053F964427FE7600A154BA3FB0030C009AA
:100D9000144B03FB1044303001F046F98DE700BFDF
:100DA0009F8601003F420F0080969800FFE0F50506
:100DB000FFC99A3B893BE65500E1F5056BCA5F6BBD
:100DC00083DE1B4340420F00C55A7C0AA086010007
:100DD0005917B7D1D34D62101F85EB51CDCCCCCC78
:080DE000834B040000CA9A3B9A
:100DE8000E4B1B68013B47F6FE72934288BF0023F7
:100DF8000A4A13600A4B1B6813B1013B084A136087
:100E0800084B1B6813B1013B064A1360064B1B686D
:100E180013B1013B044A1360704700BFC41A002095
:0C0E2800D01A0020D41A0020C01A0020AC
:100E34004FF090431A6A22F07F421A621A6822F035
:100E440070721A60144B4FF40022C3F88020BFF371
:100E54004F8FBFF36F8F4FF48012C3F88020BFF31E
:100E64004F8FBFF36F8F02F18042A2F55F22936B25
:100E740043F4000393630949B1F840309BB243F053
:100E84000203A1F84030936D23F400039365044BEF
:100E940000221A60704700BF00E100E0005C0040DF
:040EA400381A0020D8
:100EA8004F4A8023A2F84C3000214E4B1960B2F80B
:100EB80058306FEA43436FEA53439BB2A2F8583065
:100EC800A2F85010B2F850309BB203F1804303F5FA
:100ED800C043454A1360454A1360991C444A11604F
:100EE800191D444A1160991D434A116003F1080114
:100EF800424A116003F10A01414A116003F11401E9
:100F0800404A116003F116013F4A11603F4A1268D6
:100F18003AB903F118023E490A6003F11A023D4941
:100F28000A6040221A80324B1B6800221A80314B1B
:100F38001B6880211980304B1B684FF404411980CD
:100F48002E4B1B684FF4807018802D4B1B681A803D
:100F5800254B1B689881DA814FF4007018825A82F9
:100F6800284B1B681880284B1B681980274B1B6867
:100F78005BB9274B1B684FF440711980254B1B68E0
:100F88001A80194B1B689983DA83154B43F2202288
:100F98001A8043F231029A8043F232021A811B4BC3
:100FA8001B681BB90E4B43F233629A810C4B4FF40A
:100FB8003F42A3F840200023174A1360174A1360E2
:100FC800174A18490A6018490A60184A18490A60F5
:100FD80018490A60184A1370184A1370704700BFFE
:100FE800005C0040401A00203C1A0020B41A00207F
:100FF800A01A0020B81A0020A41A0020B01A002055
:101008009C1A0020AC1A0020981A0020341A0020DC
:10101800A81A0020941A0020201A0020381A00204C
:101028000C000020881A0020841A00200C080020D8
:10103800901A00208C1A00201B1800201F1A00206C
:1010480010B5254C236E43F480432366A36D43F407
:101058000003A365A36B43F40003A363FFF772F9CE
:10106800A36B23F40003A3634FF090431A6822F0A4
:1010780070721A60DA6822F07072DA60174B002119
:10108800174A23F8021B9342FBD1164B0021164A3C
:1010980023F8021B9342FBD1104CB4F858306FEA86
:1010A80043436FEA53439BB2A4F858300123A4F892
:1010B8004030C820FFF71AFA0023A4F84030A4F8FB
:1010C8004430FFF7EDFE094B4FF400221A604FF44D
:1010D80080121A6010BD00BF00100240005C004082
:1010E800205C0040445C0040605C004000E100E09F
:1010F80070B483B02E4B1B68402B50D92D4B1B6806
:1011080040221A802A4A1368403B1360294B1B6807
:101118001B88BBB1284D0022284C264E2368184650
:1011280010F8011B206058780233236041EA00233D
:1011380025F8023B013292B233681B880133B2EBC7
:10114800630FEBDB1E4B1B8813F0800F08D01C4A83
:1011580013889BB223F4E14323F070039BB21380FE
:10116800184B1B684FF404421A80154B1B889BB21E
:10117800ADF80630BDF8063013F0200F03D1104B40
:1011880048F2A0221A80BDF8063013F0100F03D1E0
:101198000B4B48F290221A8003B070BC7047044B86
:1011A8001968044A1268118000221A60AEE700BF6D
:1011B800201A0020A01A0020406000402C1A0020AD
:0811C800005C0040A41A0020A5
:1011D00082B01C4B1B6800221A801B4B1B8813F02B
:1011E000800F08D0184A13889BB223F4E14323F000
:1011F00070039BB21380134B1B6800221A80124BA2
:101200001B889BB2ADF80630BDF8063013F0200FF6
:1012100003D10D4B48F2A0221A80BDF8063013F01E
:10122000100F03D1084B48F290221A80BDF8063007
:1012300013F4804F03D0044B4CF280221A8002B08A
:0C124000704700BFA01A0020005C0040B6
:10124C0000B583B0264A13889BB223F4E14323F004
:10125C0070039BB21380234B1B68052B22D0224BAF
:10126C001B68002B38D11E4B1B8813F4004F2BD15D
:10127C001B4B1B889BB2ADF80630BDF8063013F43F
:10128C00005F03D1164B4AF280221A80BDF806305B
:10129C0013F4805F03D1124B49F280221A8003B001
:1012AC005DF804FB114B1B6843F080039BB2A2F862
:1012BC004C300C4B00221A600D4B1B68012BCED10D
:1012CC000C4BFF221A60CAE7054A138823F07003FF
:1012DC001B051B0D1380CBE7FFF708FFDFE700BFF3
:1012EC00005C0040241A0020201A0020401A002024
:0812FC00341A0020381A00200A
:1013040082B00E4B1B889BB2ADF80630BDF8063098
:1013140013F0100F03D1094B48F290221A80BDF844
:101324000630BDF8063013F4005F03D1034B4AF2D4
:1013340080221A80BDF8063002B07047005C00407D
:1013440010B586B0944B1B8813F4006F00F05581E0
:10135400914A138823F070031B051B0D13808F4BD8
:1013640093F880208E490A7093F881008D4A10709A
:10137400B3F882008C4A10801288C2F307228B488B
:101384000270B3F884008A4A1080B3F88620894B2F
:101394001A80894B00221A60884B1B684FF4044260
:1013A4001A800B78DBB2212B22D07D4B1B78DBB269
:1013B400A12B34D07A4B1B7813F0610F06D0784BF5
:1013C4001B7803F06103012B40F01481754B1B78EB
:1013D400DBB2092B00F2DC80DFE813F03A01DA001B
:1013E400DA00DA00DA0041005000DA00DA00D40052
:1013F400734B1B68002BD8D16A4B1B78DBB2202BB4
:1014040004D0684B1B78DBB2222B05D1FFF7DEFE3C
:101414006C4BFF221A601BE1FFF772FF18E1614B6E
:101424001B78DBB2212BC5D1654B1B68002BC1D1C6
:10143400614BA1221A60644A072313605D4B1B8829
:101444009BB21268934204D25A4B1B889BB25E4AE9
:1014540013605E4B5E4A1A60FFF74CFEF8E05A4B8D
:1014640000221A60FFF7B2FE4F4B1B8803F07F0384
:10147400584A1360504B05221A60E9E04E4B06228D
:101484001A604A4B1B78DBB2012B1BD0474B1B78ED
:10149400DBB2022B55D0454B1B78DBB2032B6ED14C
:1014A400494A1A231360434B1B889BB21268934228
:1014B40004D2404B1B889BB2434A1360434B464AB9
:1014C4001A602EE0404B12221A603D4B1C68434BBD
:1014D400434A012C18BF13463C4A136001AB114622
:1014E4000DF1160C0A68501C0860127803F8012BE1
:1014F4006345F7D13B4B1B6840F28342934213D0C0
:101504008DF80C301B0A8DF80D30374B1B688DF8A5
:101514000E301B0A8DF80F30012C0CD02B4B01AA76
:101524001A60FFF7E7FD93E02F4A116845F2407215
:101534009142E5D1F0E79DF80E3001338DF80E307D
:10154400ECE71F4B1B68012B12D01F4B43221A6080
:101554001E4B264A1A60174B1B889BB21A4A126804
:101564009342DED2134B1B889BB2174A1360D8E711
:10157400154B65221A60154B1D4A1A60EBE7FFF7FD
:10158400BFFE65E0104B00221A60FFF71FFE5FE00C
:10159400FFF7B6FE5CE000BF005C00400060004066
:1015A400DC1A0020DD1A00200E120020E51A0020AB
:1015B4001616002012140020241A0020A41A002059
:1015C400341A0020381A0020201A00202C1A002077
:1015D4003C3A0008401A0020683900082C390008F9
:1015E40000390008801A0020C81A0020F8390008C1
:1015F400443A0008FFF784FE2AE01A4B1B681B8854
:10160400C3F3090323BB184B1B8813F4004F21D1E8
:10161400154B1B889BB2ADF81630BDF8163013F489
:10162400005F03D1104B4AF280221A80BDF81630B5
:1016340013F4805F03D10C4B49F280221A80BDF869
:10164400163013F0400F03D0074B48F2C0221A8023
:1016540006B010BD044A138823F070031B051B0D4C
:0C1664001380D5E7A41A0020005C0040B1
:101670002DE9F04383B03B4B9B8813F0800F08D0DB
:10168000384A93889BB223F4E14323F070039BB262
:101690009380354800223549354D9646354E364CB7
:1016A0002DE0BDF80430ACF800304A46334B1B68DF
:1016B0001A802C4B9B889BB2ADF80630BDF80630E3
:1016C00013F0200F03D1274B48F2A1029A80BDF8F6
:1016D000063013F0100F03D1224B48F291029A808A
:1016E00003B0BDE8F083BDF802309AB2BDF8043013
:1016F0009BB243EA0223ACF800304A460230A0F124
:10170000020C0B68D5F800804345CFD0ADF802E05D
:1017100013F8017BADF804703768BB4208BF23465D
:101720000B6002F101095FFA89F9B9F1400FB8D0F5
:101730000B684345D7D013F8018BADF802809F4268
:1017400008BF23460B600232D2B2BDF802309FB20E
:10175000BDF804309BB243EA0723ACF80030402ABE
:10176000CCD1A3E7005C004002610040841A002055
:10177000881A0020000000200C0000209C1A002085
:1017800082B0154B9B8913F0800F08D0124A9389C1
:101790009BB223F4E14323F070039BB293810F4B80
:1017A0001B6800221A800C4B9B899BB2ADF8063057
:1017B000BDF8063013F0200F03D1074B48F2A362A7
:1017C0009A81BDF8063013F0100F03D1024B48F296
:1017D00093629A8102B07047005C0040941A002026
:1017E00010B5FEF7BDFD1F4B1C68002C33D01E4BFF
:1017F0001A681E4B1B689A4232D0511C1A4801606D
:10180000147844F400441A4A1268914225D0164ACA
:101810001268934238BF03F2FC739B1A154A126890
:10182000BAB140F2B572934213D8124B00221A603B
:10183000114B1B899AB213F4005F03D10E4B4AF28D
:101840008201198112F4805F03D10B4B49F28202AD
:101850001A81FEF76FFD204610BD08490160D6E7EA
:101860000024F8E7381A00208C1A0020901A002073
:1018700004000020281A0020005C00400C08002012
:10188000574B19684A1C1A60012800F0A38010B554
:101890000B4613F8022B524C2360022800F09C8068
:1018A00091F801C0CB1C2360032800F0978091F8C9
:1018B00002E00B1D23600438C0B2931EDBB20D2B77
:1018C00000F28B80052A2FD00F2A2DD0A2F10C0315
:1018D000DBB2012B37D902F0FB02022A51D0C978C2
:1018E000404B1A68541C1C6082F800C01A683E4BBA
:1018F0001B689A4266D03B4B1A68541C1C6082F8E5
:1019000000E01A68384B1B689A425FD0354B1A6862
:10191000541C1C6011701A68334B1B689A425CD1CE
:10192000304B324A1A6058E02E4B1A68511C19602D
:1019300082F800C01A682C4B1B689A424DD1294B83
:101940002A4A1A6049E0274B1A68511C196082F82C
:1019500000C01A68244B1B689A420ED0214B1A68AB
:10196000511C196082F800E01A681F4B1B689A42EC
:1019700033D11C4B1D4A1A602FE01A4B1B4A1A60C8
:10198000ECE71B4B00221A70164B1A68511C1960A9
:1019900082F800C01A68144B1B689A420ED0114B93
:1019A0001A68511C196082F800E01A680E4B1B6817
:1019B0009A4212D10B4B0D4A1A600EE0094B0B4AAA
:1019C0001A60ECE7074B094A1A6094E7054B074A8F
:1019D0001A609BE700207047002010BD0020FCE744
:1019E000301A0020901A0020040000200C0800206B
:0419F0001F1A00209A
:1019F40070B582B0374B1B8913F4004F11D1364BAD
:101A0400364A1A60364B1B681878364B1B6803EB52
:101A1400430290422AD9402828D82F4D324C334EC5
:101A240011E02C4A138923F070031B051B0D13814D
:101A3400E5E7FFF723FF2B4B1B6803EB43029042C0
:101A440014D9402812D8012BF3D02A68531C2B60D8
:101A54002368591C216012781A70226833689A42EC
:101A640004BF234B23600138C0B2E4E7214B1A685A
:101A74001D4B1B689A42A3EB020388BF03F2FC735D
:101A84009BB2ADF804301C4B00221A60BDF8043040
:101A94009BB240F2B672934217D80E4B1B899BB28D
:101AA400ADF80630BDF8063013F4005F03D1094BDE
:101AB4004AF282021A81BDF8063013F4805F07D11E
:101AC400044B49F282021A8102E00B4BFF221A6096
:101AD40002B070BD005C0040301A0020006200407B
:101AE400981A0020341A0020901A002004000020C4
:0C1AF4000C0800208C1A0020281A00208A
:101B000000B583B0354AB2F844309BB2ADF802302C
:101B1000B2F8443013F4004F17D1304BB3F84430CF
:101B200013F4806F47D12D4BB3F8443013F4006F9A
:101B30004DD02A4AB2F8443023F400631B041B0C36
:101B4000A2F8443003B05DF804FBBDF8023003F0A6
:101B50000F03ADF80630BDF8023003F01003ADF806
:101B60000430BDF806309BB2012B0FD0BDF8063013
:101B70009BB2022B0DD0BDF806309BB27BB9BDF8ED
:101B800004309BB243B9FFF761FBDBE7FFF770FD61
:101B9000D8E7FFF72FFFD5E7FFF7D4FBD2E7BDF873
:101BA00006309BB2032BCDD10D4B1B68002BC9D146
:101BB000FFF7E6FDC6E7FFF777F9084AB2F84430C9
:101BC00023F480631B041B0CA2F84430BAE7034BD8
:101BD00048F27F02A3F84420B4E700BF005C004055
:041BE000341A002093
:101BE40000B583B0354AB2F844309BB2ADF8023048
:101BF400B2F8443013F4004F17D1304BB3F84430EB
:101C040013F4806F47D12D4BB3F8443013F4006FB5
:101C14004DD02A4AB2F8443023F400631B041B0C51
:101C2400A2F8443003B05DF804FBBDF8023003F0C1
:101C34000F03ADF80630BDF8023003F01003ADF821
:101C44000430BDF806309BB2012B0FD0BDF806302E
:101C54009BB2022B0DD0BDF806309BB27BB9BDF808
:101C640004309BB243B9FFF7EFFADBE7FFF7FEFC62
:101C7400D8E7FFF7BDFED5E7FFF762FBD2E7BDF873
:101C840006309BB2032BCDD10D4B1B68002BC9D161
:101C9400FFF774FDC6E7FFF705F9084AB2F84430C8
:101CA40023F480631B041B0CA2F84430BAE7034BF3
:101CB40048F27F02A3F84420B4E700BF005C004070
:041CC400341A0020AE
:101CC800834A13780133DBB2137010F0800F20D1F0
:101CD800804B1B78002B00F09F807F4B1B7803F014
:101CE800F0017E4A1278002A40F0B9807C4A1070D0
:101CF8007C4A0020107003F0FD02F12A00F0958064
:101D080003F0E003C02B00F09C80744BFF221A7094
:101D18007047F72800F04881134601221A70F0280E
:101D28001BD06D4B1870F32861D900F10C03DBB29E
:101D3800012B67D9FD2865D06B4B05221A7000234B
:101D4800674A1370674A1370624A1370634A1370C4
:101D5800664A1370664A1370E1E05F4BF0221A700E
:101D68005C4BFF221A7000235C4A13705F4A1370A1
:101D78005F4A137070475C4B05221A70564BF72266
:101D88001A700023564A1370564A1370514A13703A
:101D9800524A1370554A1370554B1B781BB1544B5C
:101DA80000221A70BBE00023494A1370504A13708E
:101DB80070474D4B06221A70494B1978464A1170E4
:101DC800F7221A700023474A1370424A1370434A95
:101DD8001370464A1370464A1370A0E0444B1B78B0
:101DE800002B40F0EF803F4BF7221A70F3E0394B9D
:101DF800FF221A700023394A13703C4A13703C4A78
:101E0800137070470023334A1370344A1370374AEB
:101E18001370374A137070472D4A13702F4A137086
:101E2800324A1370324A137070472F4B02221A70CD
:101E3800284A1070294A10702C4A10702C4A1070C9
:101E48006DE00909284B1970224BFF221A700023F4
:101E5800224A1370254A1370254A13705FE0234AFB
:101E68001278002A46D11F4A1070214A12787AB98E
:101E7800F22B11D0F02B1CD009091B4B1970154BF4
:101E8800FF221A700023154A1370184A137046E08F
:101E9800164BFF221A707047134B03221A70002347
:101EA8000C4A13700D4A1370104A1370104A1370BD
:101EB80035E00D4B04221A70FF230D4A1370054AB2
:101EC80013700023054A1370084A137027E000BFF7
:101ED8001B180020DF1A0020E01A0020E41A002056
:101EE800E21A0020E11A0020DE1A0020E31A00207E
:101EF8001E1A00203D4A11783D4B19703D4B197848
:101F0800117018703C4B04221A70FF233B4A13705F
:101F18003B4A137000233B4A13703B4A13703B4BF8
:101F28001B68002B61D03A4B1A68334B1B7802F8B8
:101F3800013B384B1968384B914218BF13462C4A5D
:101F4800127803F8012B334A1168334A994218BFB3
:101F58001A46264B1B7802F8013B2E4B19682E4B6C
:101F6800914218BF1346234A127803F8012B294AD5
:101F78001168294A994208BF1346254A136000236D
:101F8800264A13701F4A13701F4A13701A4B1B7886
:101F9800072B01D8042B03D1154B1B78F02B24D920
:101FA800174B00221A707047012B3FF4E4AE022B46
:101FB8003FF4FFAE104B07221A700D4B1B78F02B25
:101FC8003FF40CAF094A1178094B1970094B19787D
:101FD8001170F7221A700023094A1370094A137006
:101FE800094A1370054A137099E77047E21A0020EE
:101FF800E01A0020E11A0020DE1A00201E1A002034
:10200800DF1A0020E41A0020E31A0020381A002002
:10201800881A0020000000200C0000201B18002057
:1020280038B5134B1B68D3B1124B1B68E3B9124B7D
:102038001A68511C196010701A68104B1B689A4274
:102048000ED00F4D0C4CFEF787F92B68226893428F
:1020580088BF02F2FC72D31AB3F5EE6FF3D838BD1D
:10206800054B084A1A60ECE7FFF72AFEF7E700BFBE
:10207800381A0020341A0020881A00200000002096
:08208800841A00200C00002066
:10209000024B4FF000629A60704700BF00ED00E015
:1020A0001D4B9B6803F00C03082B12D00C2B14D093
:1020B000042B0AD0184B9B68184AC3F30313184922
:1020C000C95C1368CB4013607047144B154A1A6003
:1020D000F0E7124B144A1A60ECE70F4BDA68DB6842
:1020E000C3F30313013302F00302022A0CBF0D49AC
:1020F0000D49B1FBF3F1084AD368D268C3F3062354
:1021000001FB03F3C2F3416201325200B3FBF2F36D
:10211000024A1360CEE700BF001002400800002012
:0C212000303700080024F40000127A00A0
:10212C0030B42C4A136E43F4804313662A4B1A685E
:10213C0022F480521A601A6842F400521A609A68AB
:10214C0022F400529A609A6842F480529A605A685B
:10215C0042F020025A6020229A611A6822F400622E
:10216C001A601A6842F480621A609A6822F400625B
:10217C009A609A6842F480629A601A6A22F07062DD
:10218C001A621A6A42F0E0621A62144BC022DA60D8
:10219C004FF400525A6000229A6009221A60104BC8
:1021AC005A1E104D104C1148114903F5007C0023A8
:1021BC0002F8013F05F8013F04F8013F00F8013F28
:1021CC0001F8013F6245F3D10A4B00221A6030BC82
:1021DC00704700BF00100240000400480038014066
:1021EC001C180020171600200F1200200B100020C6
:0821FC0013140020641A0020F6
:102204004FF4C87303494AF6AA220A60013BFCD181
:08221400704700BF00300040DC
:10221C0010B50C24FFF7F0FF631E13F0FF04F9D187
:10222C00154C4FF40013A361FFF7E6FFFFF7E4FF33
:10223C00FFF7E2FFFFF7E0FFFFF7DEFFFFF7DCFF42
:10224C00FFF7DAFFFFF7D8FF2023A361FFF7D4FFD6
:10225C000A4BDB6913F0800F08D109484AF6AA2112
:10226C00064A0160D36913F0800FFAD00023034AA9
:10227C009362044A136010BD00040048003801400A
:08228C00003000405C1A002044
:102294002DE9F043ADF5017D2A4B64221A601C46FA
:1022A400FFF79CFA50B92368002BF9D1264A136032
:1022B400264A13600DF5017DBDE8F083C3B2A22B5D
:1022C40008D0A12B23D0A02B01D1602604E001F07B
:1022D4006AFBEFE74FF400761B4BFF221A601B4B9F
:1022E4001B6813B9194B01221A60E846B1460DF177
:1022F40001031E444546134C3C272760FFF76EFA42
:1023040040B92368002BF9D101F04DFBD2E74FF41B
:102314008076E1E7C3B205F8013BB542EDD1A52BC8
:102324000DD10B490B4AC14418F8013B01F8013B9C
:1023340002F8013BC845F7D101F035FBBAE701F0DB
:1023440032FBB7E7C01A0020441A0020CC1A002040
:082354001C18002018160020DF
:10235C0008B54FF4007000F07DFD0138B0F5007F3A
:10236C0002D2034B186008BD3F20FFF757FEFAE777
:04237C00641A0020BF
:102380000D4B1A68B2B10D4B195C0D4B1B5C994299
:1023900010D08CBFCB1A5B1A1B02B3FBF2F3190AE5
:1023A000084A1154084A1354084B00221A54084B87
:1023B00001221A60704700BF581A00201C18002024
:1023C00018160020101200200C10002014140020F9
:0423D000541A00207B
:1023D40008B5094B1B6833B9084B1B68084AD0542D
:1023E400084AD05408BD054B1B68054AD05498B21E
:1023F400FFF7C4FFF6E700BF581A0020641A002054
:08240400181600201C1800202E
:10240C0008B5084B1B6840F2FF12934205D001330C
:10241C00044A1360FFF7D8FF08BD3F20FFF7FEFD0D
:08242C00FAE700BF641A00206A
:102434002DE9F041484B1D682A2D56D86C00C4F193
:10244400FF04AD000026454B1B68632B1AD8C3F16B
:102454006403C4F1FF0203FB02F24149A1FB02023F
:1024640004EB5214C5F1FF0203FB02F2A1FB0202CA
:1024740005EB5215C6F1FF0202FB03F3A1FB032394
:1024840006EB5316374B186863280FD800FB04F487
:10249400334BA3FB0424640900FB05F5A3FB0525CA
:1024A4006D0906FB00F0A3FB003046092E4FD7F858
:1024B4000080E0B2FFF78CFFE8B2FFF7A5FFF0B2AF
:1024C400FFF7A2FFC7F800802020FFF7ABFD2046EE
:1024D40001F055FA284601F052FA304601F04FFA5D
:1024E4000D20FFF79FFDBDE8F081542D0AD8A5F11A
:1024F4002B035D00AB35DC0804EB8304C4F1AA04B0
:102504000026A0E77F2D07D8A5F155004500C5F1A9
:10251400FF058600002496E7A92D0AD8803D6800AF
:1025240000F1AB06EB0803EB8505C5F1AA05002411
:1025340089E7D42D07D8A5F1AA046500C5F1FF06E3
:10254400A40000257FE7D53D6C00AB34AD00C5F198
:10255400AA06002577E700BF501A0020481A002079
:0C2564001F85EB514C1A0020641A002067
:10257000F8B12DE9F8430F4BD3F800900E4B13F848
:10258000098086B200250B4C40F2FF172368013307
:1025900023604046FFF71EFF2368BB4203D001358E
:1025A000ABB2B342F2D31FFA89F3024A1360BDE81B
:0C25B000F8837047641A00201816002001
:1025BC002DE9F04F0020204B1860204B5A1E204F65
:1025CC00204E214C214D03F2FF1A84464FF0010B93
:1025DC000DE0A3EB0C039942C8BF0BB28EF8003090
:1025EC00DC46FF2001360134013552451DD0013245
:1025FC009646137817F8011F8B42F3D096F800C05B
:10260C00207895F8008000EB080984F80090484683
:10261C00FF2884BF0CF1010C5FFA8CFC8B42D8D2E2
:10262C0063449942DADA0BB2D8E7BCF1000F01D05F
:10263C00014B1860BDE8F08F541A00201C180020C4
:10264C001716002010120020141400200C1000206B
:10265C0008B50E4B1A680E4B1A600E4B1B680E4ACF
:10266C0010681844DC2802D9002111601846FEF7C6
:10267C0067F8094A136801331360084A12689342D9
:10268C0000D008BD044B00221A60FAE7681A00203B
:10269C00781A0020701A00206C1A0020741A00207E
:1026AC0070B590B00646824B0CAC0FCB07C42370B0
:1026BC00804B08AC0FCB07C423707F4B93E803000F
:1026CC000690ADF81C10090C8DF81E1001AC7B4D5A
:1026DC000FCD0FC42B6823603546002E40F0A08030
:1026EC000CA801F03EFA764C2068013001F043F959
:1026FC005420FFF793FC7820FFF790FC3A20FFF76B
:10270C008DFC23686F4AD05C01F035F906A801F006
:10271C0028FA23686C4AD05C01F02DF92020FFF7D1
:10272C007DFC2820FFF77AFC684801F01AFA684E05
:10273C0034686848A0FB0434C4F307142046FEF741
:10274C0099FA2E20FFF76AFC3068634BA3FB00302C
:10275C0004EB84046400C4EB9000FEF78BFA732046
:10276C00FFF75CFC2020FFF759FC2020FFF756FCFC
:10277C005A4801F0F6F95A4B1868FEF77BFA2920F3
:10278C00FFF74CFC002D4FD00D20FFF747FC4C4BB6
:10279C001B68B3F5FF7F4AD208A801F0E2F9484C58
:1027AC002068023001F0E7F85420FFF737FC78205E
:1027BC00FFF734FC3A20FFF731FC424E23683344D8
:1027CC00587801F0D8F806A801F0CBF93E4D2368F3
:1027DC002B44587801F0CFF80D20FFF71FFC08A808
:1027EC0001F0BFF92068033001F0C5F85420FFF761
:1027FC0015FC7820FFF712FC3A20FFF70FFC23683A
:10280C001E44B07801F0B7F806A801F0AAF92368C5
:10281C001D44A87801F0AFF80D20FFF7FFFB06E090
:10282C000D20FFF7FBFB5BE72020FFF7F7FB01A870
:10283C0001F097F92B4B186801F09DF84C20FFF72D
:10284C00EDFB6520FFF7EAFB6E20FFF7E7FB3A2074
:10285C00FFF7E4FB244B186801F08DF85320FFF7C9
:10286C00DDFB7420FFF7DAFB6520FFF7D7FB702048
:10287C00FFF7D4FB3A20FFF7D1FB1C4D2868164C10
:10288C00A4FB0030C008FEF7F5F92E20FFF7C6FBBD
:10289C002868A4FB0034E40804EB8404A0EB440097
:1028AC00C0B201F030F87320FFF7B8FB10B070BD68
:1028BC0040370008503700086037000868370008B8
:1028CC00641A00201C18002018160020383B000841
:1028DC00581A00201F85EB51CDCCCCCCC039000848
:1028EC00601A0020701A0020741A0020681A002048
:1028FC00F8B50D4668BB5320FFF790FB1E4C2068C3
:10290C000130FEF7B7F93A20FFF788FB5620FFF7A6
:10291C0085FB3D20FFF782FB2488184B185DFEF7E2
:10292C00A9F90134A4B2013DB4F5007F10D07DB1FA
:10293C002C27124E3846FFF771FB305DFEF79AF9E3
:10294C000134A4B2013DB4F5007F01D0002DF1D1CA
:10295C00F8BD2020FFF762FB6620FFF75FFB7220BB
:10296C00FFF75CFB6F20FFF759FB6D20FFF756FB61
:10297C002020FFF753FBBEE7641A00201C18002030
:10298C0038B50446084B187840F0B000FFF746FB0A
:10299C00064D285D00F001005430FFF73FFB285D29
:1029AC004008FFF73BFB38BDD81A00201C1800204C
:1029BC0070B5194B1B6840F2FF12934228D05D1C76
:1029CC00ED095035EDB2013303F07F04134E30782E
:1029DC0040F0B000FFF722FB2846FFF71FFB204614
:1029EC00FFF71CFB307840F0B000FFF717FB01201D
:1029FC00FFF714FB0A4B18680A4BA3FB0030C0F31B
:102A0C008700FFF70BFB044B1888FFF7B9FF70BD6D
:102A1C0000245025DAE700BF641A0020D81A0020E1
:082A2C00581A0020CDCCCCCCDF
:102A34002DE9F041A84C00252560082800F0E1812B
:102A44001E4601F00F01092800F0DE81A34B1B682C
:102A5400994240F0D481A0F1090CBCF1050F00F2B9
:102A6400CE81DFE81CF0D801CC0127006501CC0140
:102A7400C3019A4B1B68C91A02EBC112984B1A6026
:102A84001AB9974B4FF400721A60954A1368013BC8
:102A940013607300DEB2FE2E07D0022E06D1914BD6
:102AA4001B68002B08BF002600E0FF263046FFF716
:102AB4008FFCA4E1012A0DD0A2F15003DBB2032B59
:102AC40012D8502A0BD0503A06EBC213013B844A69
:102AD400136094E106EB8606834A16608FE1002EAC
:102AE400F1D14FF40073F1E7542A35D0552A39D087
:102AF400562A3DD0572A4AD0102A57D0122A5AD0E3
:102B0400132A6CD0142A72D0242A7ED0252A00F0ED
:102B1400AB80282A00F0B980302A00F0BA80402A1D
:102B240000F0BF80412A00F0C280422A00F0C78032
:102B3400602A00F0CC80612A00F0EC80702A00F05A
:102B4400F080712A40F0F1805C2E00F2588106F189
:102B54008000FDF7D5FF52E1700000F0FE00FFF7A2
:102B640037FC4CE17300581CC0B2FFF731FC46E15E
:102B74005B4B1B68B3F5FF7F00F241810133584A78
:102B84001360700000F0FE00FFF722FC37E1544BA5
:102B94001B68B3F5FF7F00F232810133504A1360A2
:102BA4007300581CC0B2FFF713FC28E14F4B1E60A2
:102BB4004F4B1E6023E1012E0AD94E4B1E604E4B33
:102BC4001B689E4200F21B814B4B00221A6016E1E7
:102BD4003F20FFF727FA494B00221A70EDE7484BD4
:102BE4001E60454B00221A60FFF736FD07E13346AD
:102BF4005C2E28BF5C2383F08003414A13603E4B64
:102C040000221A60FFF728FDF9E0002E00F0F7809B
:102C1400FFF7D2FE012E00F0F280013EF6B2304BF7
:102C24001A6893B25C1CA4B2092E28BF0926324448
:102C3400944200F2E480B4F5007F00F2E0800233B5
:102C44009DB2DFF89C8040F201272046FFF79CFEEE
:102C54000134A4B2D8F800303344AB42C0F0CF8082
:102C64000135BC42F1D1CAE0002E00F0C880F0204A
:102C7400FFF7D8F97D20FFF7D5F931460020FFF79B
:102C84003BFEF720FFF7CEF9B9E03046FFF76EFCC4
:102C9400B5E0042E40F2B380731C9B00194A136004
:102CA400ADE07600184A1660FFF7C2FBA7E0642E79
:102CB40028BF6426154A1660FFF7BAFB9FE0642E0E
:102CC40028BF6426124A1660FFF7B2FB97E030462D
:102CD400FDF73AFD93E000BFCC1A0020D81A00207B
:102CE400641A00207C1A0020581A0020681A002058
:102CF400781A0020741A00206C1A0020E61A0020AA
:102D0400701A0020601A0020501A0020481A00206F
:102D14004C1A00205C2E72D806F18000FDF714FDD9
:102D24006DE03046FDF7ECFE69E0772A67D1324664
:102D3400012A0FD0082A1BD0092A27D0102A33D001
:102D4400772A34D0782A3FD0792A41D13B4BFF22CD
:102D54001A6054E03A4B1968002950D00023394CCA
:102D64003948C25CE25401339BB28B42F9D346E04A
:102D7400364B1B68344AD25C002A40D0013A3249AF
:102D8400CA543049CA5C013ACA5438E02F4B1B6814
:102D94002D4AD25CFF2A32D001322B49CA54294928
:102DA400CA5C0132CA542AE0FFF756FC27E0F0203F
:102DB400FFF738F97D20FFF735F90020FFF774FCA1
:102DC400F720FFF72FF91AE01C4B00221A6016E0D7
:102DD4007F2A14D11E4B1F4903F50070002203F80B
:102DE400012F01F8012F8342F9D108E07300D8B212
:102DF40012F0400F1CBF0130C0B2FFF7E9FABDE882
:102E0400F08101F00F010026134B1B689942F6D3A1
:102E140003339942F3D8002E7FF42BAE074B1B6883
:102E2400002BECD00C4B1B68C91A12EBC1123FF4F7
:102E340028AE013A054B1A6038E600BF7C1A002020
:102E4400601A0020181600201C180020641A0020A4
:0C2E54001B18002017160020D81A0020C0
:102E600070B5184B984225D806460024FEF7B8FCEA
:102E700083B2002BFAD0C0B21B281FD00A281BD067
:102E80000D2819D02E2817D0A0F13005EDB2092D4C
:102E90000DD8FFF7C9F804EB840405EB4404A642FF
:102EA000E4D23F20FFF7C0F84FF0FF3404E0064BB8
:102EB000187001E04FF0FF34204670BD4FF0FF3432
:0C2EC000FAE700BFB7820100E61A00200C
:102ECC002DE9F04F85B0424B93E8030002908DF84A
:102EDC000C10404B93E8030000908DF8041002A8EE
:102EEC0000F03FFE00F049FEFF2804D900242046E4
:102EFC0005B0BDE8F08F044600F03FFE0546FF2804
:102F0C0001D90024F3E700F038FE0646FF2801D96A
:102F1C000024ECE700F031FE0746FF2801D900241D
:102F2C00E5E72020FFF77AF8684600F01AFE00F07B
:102F3C0024FE8046FF2801D90024D8E700F01DFEAE
:102F4C008146FF2801D90024D1E700F016FE824605
:102F5C00FF2801D90024CAE700F00FFE8346FF28A2
:102F6C0001D90024C3E70D20FFF758F81A4800F0E8
:102F7C00F8FDFEF72FFC0028FBD048F259029042D6
:102F8C0001D00124B3E705EB041406EB041407EBA2
:102F9C000414124B1C6009EB08180AEB08180BEB15
:102FAC0008180F4BC3F800800120FDF703FB044603
:102FBC0050B12020FFF732F86F20FFF72FF86B206D
:102FCC00FFF72CF8012492E7064800F0CAFD8EE7C3
:102FDC00AC3A0008B43A0008F83A0008801A00200D
:082FEC00C81A0020243B000874
:102FF40010B582B0194B93E8030002AB03E9030058
:103004001020FFF72BFF441E0F2C04D9684600F054
:10301400ACFD02B010BD0D20FFF704F8104800F01D
:10302400A4FDFEF7DBFB0028FBD048F259029042D6
:10303400EFD10C4B1C600120FDF7C0FA48B12020F1
:10304400FEF7F0FF6F20FEF7EDFF6B20FEF7EAFFBF
:10305400DFE7054800F089FDDBE700BF7C370008A7
:0C306400F83A0008D81A0020243B0008AD
:1030700030B595B00FAC414D0FCD0FC42B6824F87F
:10308000023B1B0C23700DF1180C3D4C0FCCACE82F
:103090000F000FCCACE80F002368CCF800306C4672
:1030A000384D0FCD0FC495E8030084E803000D20D0
:1030B000FEF7BAFF06A800F05AFD3220FEF7B4FF73
:1030C0002E20FEF7B1FF3520FEF7AEFF684600F078
:1030D0004EFD0D20FEF7A8FF0FA800F048FD0D20C3
:1030E000FEF7A2FF284800F042FD284D2C68284832
:1030F000A0FB0434C4F307142046FDF7C1FD2E20C5
:10310000FEF792FF2868234BA3FB003004EB8404F6
:103110006400C4EB9000FDF7B3FD7320FEF784FF5D
:103120000D20FEF781FF1C4800F021FD1B4B1868A5
:10313000FDF7A6FD0D20FEF777FF194800F017FDFB
:10314000184B186800F00F00013000F052FD0D2000
:10315000FEF76AFF144800F00AFD144B188800F0CF
:10316000EEFB2F20FEF760FF2020FEF75DFF104BE7
:10317000188800F0E4FB15B030BD00BF84370008AC
:1031800098370008BC370008383B0008581A002060
:103190001F85EB51CDCCCCCCC0390008601A002083
:1031A00090390008D81A00204C3B0008801A0020F3
:0431B000C81A002019
:1031B40030B591B004460DF1200C904D0FCDACE824
:1031C4000F0095E80F00ACE807002CF8023B1B0C3D
:1031D4008CF800300DF1040C894D0FCDACE80F00D4
:1031E40095E80700ACE803008CF80020854B00222A
:1031F4001A60A4F16103DBB2192B05D8203CE4B2B8
:103204002046FEF70FFF01E0202CF9D80A3C742C6D
:1032140000F25D82DFE814F04D025B025B025402AF
:103224005B025B025B025B025B025B025B025B02B2
:103234005B025B025B025B025B025B025B025B02A2
:103244005B025B0284005B025B025B025B025B026B
:103254005B025B025B025B025B02D5009C00E30045
:103264005B025B025B025B025B025B025B025B0272
:103274005B025B025B025B025B025B025B0241017D
:103284005B02470223029A0164010B02E4015B0220
:103294005B02860153015B025B025B02D1015B02AC
:1032A400CE015B02BD01AC00B0008200C400140278
:1032B4008C00750175005B025B025B025B025B02C2
:1032C400040121015B025B025B025B025B025B02A5
:1032D4005B025B025B025B025B025B025B025B0202
:1032E4005B025B025B025B025B025B025B025B02F2
:1032F4005B025B025B025B025B025B025B025B02E2
:103304003202414B186858B1404B414A184413F8F3
:10331400011B02F8011B8342F9D101E0FFF71CF8FD
:103324000D20FEF77FFE3E20FEF77CFE11B030BD7F
:10333400FF20FFF793FDFF2806D93F20FEF772FE1A
:10334400344B00221A70EBE7C0B2FFF741F8E7E70D
:10335400FF20FFF783FDFF2806D93F20FEF762FE1A
:103364002C4B00221A70DBE7C0B2FFF74DF8D7E709
:103374000120FFF799F9D3E701A800F0F6FB4FF419
:103384000070FFF76BFD0146431EB3F5007F03D2C7
:103394000120FFF7B1FAC3E73F20FEF743FEC5E77C
:1033A4007F20FFF75BFD7F2804D800EB80001A4BD9
:1033B4001860B5E73F20FEF735FE164B00221A7061
:1033C400AEE7164B1B68114AD25CFF2AA8D0013223
:1033D4000E49CA540E49CA5C0132CA54A0E70F4BC5
:1033E4001B680A4AD25C002A9AD0013A0749CA5497
:1033F4000749CA5C013ACA5492E700BFBC3A0008C4
:10340400DC3A0008CC1A0020601A00201C180020A6
:1034140018160020E61A0020581A0020641A00200A
:10342400FF20FFF71BFD0446FF280FD8AB4B1A689B
:10343400AB48815C0C44FF2C28BFFF24E3B2194441
:103444008154A849885C03448B5469E73F20FEF704
:10345400E9FDA54B00221A70E8E7FF20FFF7FEFC08
:103464000446FF2812D89D4B1A689D4B995C0B1B90
:103474004FF6FE70834288BF0023DBB2C91A984816
:1034840081549848815CCB1A835449E73F20FEF766
:10349400C9FD954B00221A70E5E740F2FF10FFF7D3
:1034A400DDFCB0F5007F06D33F20FEF7BBFD8E4B5D
:1034B40000221A7034E7C0B2FFF758F830E7FF2053
:1034C400FFF7CCFCFF2806D93F20FEF7ABFD864B67
:1034D40000221A7024E7854B1860FEF7A9FF1FE746
:1034E4006420FFF7BBFC642806D93F20FEF79AFD51
:1034F4007D4B00221A7013E77D4B1860FEF798FF8E
:103504000EE76420FFF7AAFC642806D93F20FEF7E3
:1035140089FD754B00221A7002E7764B1860FEF79E
:1035240087FFFDE6DC20FFF799FCDC2806D93F2065
:10353400FEF778FD6C4B00221A70F1E66E4B1860B2
:103544006E4B00221A60FFF787F8E9E6DC20FFF7EC
:1035540085FCDC280CD8012811D0694B186001289F
:1035640002D9684B02221A60644B00221A60D7E623
:103574003F20FEF757FD5C4B00221A70D0E63F2037
:10358400FEF750FD584B00221A705D4B01221A6061
:10359400EAE7FF20FFF762FCFF2804D85A4B1860C3
:1035A400584B1860BCE63F20FEF73CFD4E4B002212
:1035B4001A70B5E6FFF750F8B2E64FF40070FFF763
:1035C4004DFCA0F11803B3F5F47F02D84F4B1860FB
:1035D400A6E63F20FEF726FD434B00221A709FE625
:1035E4000D20FEF71FFD08A800F0BFFA4FF4FA7093
:1035F400FCF77EFFFEF7F2F80028FBD020F0200352
:1036040048F24402934206D03F20FEF70BFD364BAE
:1036140000221A7084E63E4B3E4903F500700022F6
:1036240003F8012F01F8012F8342F9D178E63A48D3
:1036340000F09BFA394800F098FAFFF7D9FC6FE6DE
:10364400354800F092FA364800F08FFAFFF73CFC58
:1036540000287FF465AE3F20FEF7E4FC60E6DC2042
:10366400FFF7FCFBDC2806D93F20FEF7DBFC1E4BF2
:1036740000221A7054E6FDF767F851E6DC20FFF7E4
:10368400EDFBDC2806D93F20FEF7CCFC164B0022CC
:103694001A7045E6FDF734FA00287FF441AE21485C
:1036A40000F063FA3CE6204B00221A60FFF7DEFCD0
:1036B40036E60D20FEF7B6FC3E20FEF7B3FC35E6F9
:1036C4000D20FEF7AFFC3E20FEF7ACFC2EE63F20BB
:1036D400FEF7A8FC044B00221A7021E6641A0020AD
:1036E4001C18002018160020E61A0020501A00208A
:1036F4004C1A0020481A0020701A00206C1A00206E
:10370400741A0020781A0020681A0020601A002019
:103714001B18002017160020443B000890390008AD
:0C3724004C3B0008243B0008BC1A0020AD
:103730000000000000000000010203040607080961
:10374000444D58206368616E6E656C3A000000005D
:10375000202020206368616E6E656C3A00000000D6
:1037600046696E616C3A000043686173657220536C
:0C37700074617274205363656E653A004A
:08377C0020312D3136213F0000
:10378400476C6F62616C20706172616D6574657203
:10379400733A00005553422F444D5820436F6E74C2
:1037A400726F6C6C657220776974682053544D3362
:1037B40032473433312076002028632932303230C6
:1037C4002D323120572E536368656D6D6572740018
:1037D400FEE7FEE7FEE7FEE7FEE7FEE7FEE7FEE7BD
:1037E400FEE7FEE7FEE7FEE7FEE7FEE7FEE7FEE7AD
:1037F400FEE7FEE7FEE7FEE7FEE7FEE7FEE7FEE79D
:10380400FEE7FEE7FEE7FEE7FEE7FEE7FEE7FEE78C
:10381400FEE7FEE7FEE7FEE7FEE7FEE7FEE7FEE77C
:10382400FEE7FEE7FEE7FEE7FEE7FEE7FEE7FEE76C
:10383400FEE7FEE7FEE7FEE7FEE7FEE7FEE7FEE75C
:10384400FEE7FEE7FEE7FEE7FEE7FEE7FEE7FEE74C
:10385400FEE7FEE7FEE7FEE7FEE7FEE7FEE7FEE73C
:10386400FEE7FEE7FEE7FEE7FEE7FEE7FEE70348C6
:103874008546FEF70BFC00F003B87047008000207B
:1038840011488546114C20680434004201D0804719
:10389400F9E70F480F49091A082903DB00220260DF
:1038A400043001600C480D49884205D00268043098
:1038B40003B4904703BCF7E700208646EC4600209B
:1038C4000021074A9047FEE7008000200C3C0008D6
:1038D400E81A0020E81E00203B3A00083B3A0008A2
:0438E4004908000887
:1038E8001EF0040F0CBFEFF30880EFF309800149C5
:0838F80008470000D339000865
:10390000120100020000004083044057050200013C
:023910000001B4
:1039120008B5024600F13003D8B2392884BF02F15B
:0A3922003700C0B2FEF77FFB08BDBE
:10392C00120100020000004083044157050200010F
:02393C00000188
:10393E0010B50446000BFFF7E5FFC4F30320FFF7B5
:10394E00E1FFC4F30310FFF7DDFF04F00F00FFF7F4
:0A395E00D9FF2020FEF761FB10BD29
:103968001A035500530042002F0044006D007800F0
:0A39780020004300740072006C0090
:0E39820008B5FDF77CF92020FEF74DFB08BDCF
:103990004D4944492062617365206368616E6E65BC
:0A39A0006C2028312D3136293A0041
:1039AA0008B55A20FEF73BFBC120FEF738FBA520DD
:0639BA00FEF735FB08BD1D
:1039C000444D58206379636C65206C656E6774683C
:0239D0003A00BB
:1039D2004FF0E023D3F82C3D002B00DBFEE74FF045
:1039E200E022D2F82C3D43F00043C2F82C3D83691B
:0639F200023383617047FF
:1039F80009024300020100803109040000010202AB
:103A08000000052400100105240103000424020716
:103A1800052406000107058303100040090401007E
:103A2800020A0000000705810240000007050202A3
:033A38004000004B
:073A3C0000C20100000008B8
:103A4400090265000201008031090400000001013F
:103A54000000092401000109000101090401000218
:103A640001030000072401000141000624020101B2
:103A740000062402020200092403010301020100DA
:103A84000924030204010101000905810240000028
:103A940000000525010103090502024000000000A1
:053AA4000525010101F0
:0D3AAC005669643D000000005069643D0053
:103ABC00616C6C206C6967687473204441524B3F95
:103ACC002D3E707265737320616761696E20000012
:103ADC0065616420686F77206D616E7920444D5864
:093AEC00206C6576656C733F00E7
:103AF8005361766520536574757020746F20466C29
:103B08006173683F2D3E70726573732075707065C0
:0B3B18007220636173652027592700AD
:103B2400466C617368205772697465204572726FC0
:023B340072001D
:0A3B38004661646574696D653A002A
:063B4400202073657400EF
:103B4C00555342205669642F506964206F66207467
:103B5C0068697320646576696365202868657829CF
:023B6C003A001D
:103B6E0010B5044614F8010B28B1FEF756FA14F8F6
:083B7E00010B0028F9D110BD74
:103B860038B5FDF72AFE83B2002BFAD0C4B21B2C3F
:103B960020D00A2C21D00D2C22D02E2C23D0A4F1FB
:103BA6003005092D0CD9A4F16103192B98BF203CCF
:103BB600A4F14103052B07D94FF0FF35284638BD40
:103BC6002046FEF72EFAF9E7E0B2FEF72AFAA4F14C
:103BD6003705F3E74FF0FF35F0E76FF00105EDE746
:0C3BE6006FF00105EAE76FF00105E7E76A
:103BF20010B50446092803D92046FFF7C1FE10BDBF
:083C02002020FEF710FAF7E79D
:103C0C00393C00080C000020DC1A00004F3C000876
:103C1C00000000202C3C00080C00000000000000FC
:0C3C2C0008080020081000200024F4000C
:103C3800206861680834094204D00022027001300B
:063C48000139FBD17047B9
:103C4E0020686168A2680C34124205D00B780370AC
:0A3C5E0001300131013AF9D170473D
:040000050800387344
:00000001FF
